S02800002E2E5C62696E5C64656D6F70726F675F6F6C696D65785F73746D3332703430352E7372656344
S3150800800000000220258D0008738D0008758D000874
S31508008010778D0008798D00087B8D00080000000028
S315080080200000000000000000000000007D8D000830
S315080080307F8D000800000000818D0008898E0008E9
S31508008040878D0008898D00088B8D00088D8D0008A6
S315080080508F8D0008918D0008938D0008958D000876
S31508008060978D0008998D00089B8D00089D8D000846
S315080080709F8D0008A18D0008A38D0008A58D000816
S31508008080A78D0008A98D0008AB8D0008AD8D0008E6
S31508008090AF8D0008B18D0008B38D0008B58D0008B6
S315080080A0B78D0008B98D0008BB8D0008BD8D000886
S315080080B0BF8D0008C18D0008C38D0008C58D000856
S315080080C0C78D0008C98D0008CB8D0008CD8D000826
S315080080D0CF8D0008D18D0008D38D0008D58D0008F6
S315080080E0D78D0008D98D0008DB8D0008DD8D0008C6
S315080080F0DF8D0008E18D0008E38D0008E58D000896
S31508008100E78D0008E98D0008EB8D0008ED8D000865
S31508008110EF8D0008F18D0008F38D0008F58D000835
S31508008120F78D0008F98D0008FB8D0008FD8D000805
S31508008130FF8D0008018E0008038E0008058E0008D2
S31508008140078E0008098E00080B8E00080D8E0008A1
S315080081500F8E0008118E0008138E0008158E000871
S31508008160178E0008198E00081B8E00081D8E000841
S315080081701F8E0008218E0008238E0008258E000811
S31508008180278E0008298E0008EE11AA5510B5054C51
S31508008190237833B9044B13B10448AFF300800123A5
S315080081A0237010BD7C00002000000000648F0008CA
S315080081B0084B10B51BB108490848AFF300800848BA
S315080081C0036803B910BD074B002BFBD0BDE8104070
S315080081D0184700BF0000000080000020648F0008D8
S315080081E07C00002000000000154B002B08BF134B35
S315080081F09D46A3F5803A00218B460F461348144A3C
S31508008200121A00F083FE0F4B002B00D098470E4B36
S31508008210002B00D098470020002104000D000D48CF
S31508008220002802D00C48AFF3008000F049FE200079
S31508008230290000F06DFD00F02FFE00BF00000800C9
S315080082400000022000000000000000007C00002062
S31508008250F00000200000000000000000F0B5002437
S3150800826021E0134D15F8147005EB440595F801E067
S3150800827007EB0E0505FB00054AF2104C9CFBF5F6CC
S3150800828005FB16C66EB99CFBF5F5ADB20D80013D32
S31508008290ADB2B5F5806F04D2177083F800E00120FF
S315080082A0F0BD0134E4B2112CDBD90020F0BD00BFCB
S315080082B0388F0008F0B587B001214FF4003000F080
S315080082C0FBFB0121084600F0E9FB1E4D07220221AF
S315080082D0284600F06FFB07220321284600F06AFBB8
S315080082E000248DF8164001278DF8177002268DF8A0
S315080082F01460042304938DF8156004A9284600F039
S3150800830013FB8DF814600823049304A9284600F08B
S315080083100BFB4FF461430093ADF80440ADF80640FB
S31508008320ADF80840ADF80C400C23ADF80A30064C01
S315080083306946204600F0DCFB3946204600F040FC42
S3150800834007B0F0BD000002400044004070B58AB096
S315080083500121022000F0A2FB354E092208213046F1
S3150800836000F028FB09221146304600F023FB4FF4A3
S315080083704073089302238DF824308DF825300024A5
S315080083808DF8264001258DF8275008A9304600F0BB
S31508008390CBFA29464FF0007000F08EFBA6F5D036D2
S315080083A0304600F031F905A800F04CFA6B460DEBA3
S315080083B005020DF102014FF4FA70FFF74FFF8DF831
S315080083C01A408DF81B408DF81C408DF81D408DF81D
S315080083D01E408DF81F408DF816408DF817409DF801
S315080083E00130013B8DF818309DF80030013B8DF8BF
S315080083F01930BDF80230ADF8143005A9304600F042
S315080084001FF98DF80E408DF80F408DF81050ADF815
S315080084100440ADF80640ADF80840ADF80A40ADF89E
S315080084200C408DF8115001A800F092F90AB070BD01
S315080084300004024010B504462021064800F0D2FB8D
S31508008440012805D1034800F0C9FB2070012010BDA2
S31508008450002010BD0044004008B5FFF72BFFFFF7CA
S3150800846075FF08BDBFF34F8F0449CA6802F4E0627E
S31508008470034B1343CB60BFF34F8FFEE700ED00E0DD
S315080084800400FA0508B5204B1B789BB91F48FFF76F
S31508008490D1FF012836D11D4B1B78002B32D000F0B6
S315080084A0EDFC1B4B18600122174B1A700022194B62
S315080084B01A7008BD174B1B78013314481844FFF788
S315080084C0B9FF012814D1134A13780133DBB21370AC
S315080084D00E4A1278934215D100220B4B1A700B4B99
S315080084E05B78FF2B0ED1094B9B785BB9FFF7BAFF78
S315080084F000F0C4FC064B1B686433984202D900227C
S31508008500014B1A7008BD00BFE1000020A000002042
S31508008510980000209C00002000B587B00021114873
S3150800852000F0F4F9D8B101AA00210E4800F09AF932
S315080085309DF80C3033B940F26763019A9A4203D02A
S31508008540002302E0002300E0012343B19DF80F3029
S31508008550FF2B04D19DF810300BB9FFF783FF07B046
S315080085605DF804FB0064004008B5FFF78BFFFFF7D2
S31508008570D3FF08BD30B583B00121042000F08EFA80
S315080085804FF48055009501238DF8043000228DF8AC
S3150800859006208DF8073002238DF80530054C69460C
S315080085A0204600F0C1F92946204600F0FFF903B03D
S315080085B030BD00BF0008024010B500F05FFC0F4B4D
S315080085C01B68C31AB3F5FA7F16D304460C4B1B78FF
S315080085D043B901220A4B1A704FF48051094800F03A
S315080085E0E7F907E00022064B1A704FF48051054858
S315080085F000F0DCF9014B1C6010BD00BFE400002050
S31508008600E80000200008024008B50C4B98420AD141
S3150800861001214FF0007000F05DFA00214FF0007064
S3150800862000F058FA08BD01214FF0806000F052FAB8
S3150800863000214FF0806000F04DFA08BD006400404C
S31508008640036823F002030360036843F00103036031
S31508008650002300E00133426812F0010F03D14FF600
S31508008660FF729342F6D1436813F0010F6BD08B79F2
S31508008670012B04D1036843F08003036003E0036819
S3150800868023F080030360CB79012B04D1036843F000
S315080086904003036003E0036823F0400303600B7A9A
S315080086A0012B04D1036843F02003036003E0036849
S315080086B023F0200303604B7A012B04D1036843F0AF
S315080086C01003036003E0036823F0100303608B7A4A
S315080086D0012B04D1036843F00803036003E0036831
S315080086E023F008030360CB7A012B04D1036843F017
S315080086F00403036003E0036823F0040303608A7835
S31508008700CB781B0643EA82730A7943EA02434A791D
S3150800871043EA02530A88013A1343C361036823F004
S3150800872001030360002300E00133426812F0010FE1
S3150800873003D04FF6FF729342F6D1436813F0010F48
S3150800874003D000207047002070470120704700BF03
S3150800875070B4837A012202FA03F3394AD2F8001276
S3150800876041F00101C2F80012D2F81C12DC43214084
S31508008770C2F81C12027BB2B9314AD2F80C12214057
S31508008780C2F80C12817AC688458845EA06454831FA
S3150800879042F83150857A8688018841EA064148358B
S315080087A002EBC5025160027B012A16D1244AD2F88F
S315080087B00C121943C2F80C12817A0688458845EAD4
S315080087C00645483142F83150857A8688C18841EA9B
S315080087D00641483502EBC5025160C27A32B91849DA
S315080087E0D1F804222240C1F8042205E01449D1F840
S315080087F004221A43C1F8042202892AB91049D1F879
S3150800880014221440C1F814420289012A05D10C49E0
S31508008810D1F814221A43C1F81422427B012A05D141
S315080088200749D1F81C221343C1F81C32044AD2F86E
S31508008830003223F00103C2F8003270BC704700BF53
S315080088400064004000238371C3710372437283720C
S31508008850C3728370C3700323037102234371012318
S315080088600380704710B401F11B031B01C35803F0C2
S315080088700403DBB2137233B901F11B031B01C3589E
S315080088805B0D136005E001F11B031B01C358DB08F0
S31508008890536001F11B031B01C418C35803F00203FC
S315080088A05372636803F00F03937263681B0AD374E9
S315080088B000EB0113D3F8B841D472D3F8B841240AAF
S315080088C01473D3F8B841240C5473D3F8B841240E62
S315080088D09473D3F8BC41D473D3F8BC41240A1474F6
S315080088E0D3F8BC41240C5474D3F8BC311B0E9374D2
S315080088F021B9C36843F02003C36003E0036943F06A
S31508008900200303615DF8044B704700BF19B9C068BE
S3150800891000F003007047012903D1006900F0030045
S3150800892070470020704700BF70B400233AE0012268
S315080089309A400C68A24334D104685D000322AA4019
S31508008940D2431440046006680C79AC403443046092
S315080089500C79013CE4B2012C15D884682240826067
S3150800896084684A79AA402243826046689AB20124FA
S31508008970944026EA0404446046688C7904FA02F2B4
S3150800898092B232434260C4689AB256000322B24099
S3150800899024EA0202C260C668CC7904FA05F23243B8
S315080089A0C26001330F2BC2D970BC70470183704770
S315080089B04183704730B401F007039B009A40C90809
S315080089C0083150F821400F2505FA03F324EA03037A
S315080089D040F8213050F821301A4340F8212030BCA5
S315080089E0704700BF10B4294B9B6803F00C03042B97
S315080089F005D0082B06D053BB254B036029E0254B31
S31508008A00036026E0214B5A685B6803F03F0312F4C3
S31508008A10800F09D01F4AB2FBF3F21C4B5B68C3F305
S31508008A20881303FB02F208E0194AB2FBF3F3174A6C
S31508008A305168C1F3881101FB03F2144B5B68C3F359
S31508008A40014301335B00B2FBF3F3036001E0104B13
S31508008A5003600E4CA368C3F303130F49CB5CDAB269
S31508008A600368D3404360A268C2F382228A5CD2B20A
S31508008A7023FA02F28260A268C2F342328A5CD2B258
S31508008A80D340C3605DF8044B704700BF003802400E
S31508008A900024F40000127A000000002021B1054BE2
S31508008AA01A6B104318637047024A136B23EA0000D7
S31508008AB0106370470038024021B1054B1A6C104309
S31508008AC018647047024A136C23EA00001064704762
S31508008AD00038024021B1054B1A6A104318627047E4
S31508008AE0024A136A23EA00001062704700380240FF
S31508008AF030B585B004460D46038A9BB223F440532D
S31508008B00CA881343038283899BB223F4B05323F0A4
S31508008B100C01A8882A896B89024313430B43A38156
S31508008B20A38A9BB223F44073AA891343A382684697
S31508008B30FFF758FF204B9C4203D003F580639C4205
S31508008B4001D1039A00E0029AA38913F4004F08D0D2
S31508008B5002EB820202EB820229684900B2FBF1F1BC
S31508008B6007E002EB820202EB820229688900B2FB67
S31508008B70F1F1124BA3FB01235B091B011A096420BF
S31508008B8000FB1212A18911F4004F08D0D20032322C
S31508008B900A49A1FB0212C2F342121A4307E0120164
S31508008BA032320649A1FB0212C2F343121A4392B2A9
S31508008BB0228105B030BD00BF001001401F85EB5172
S31508008BC029B183899BB243F4005383817047838913
S31508008BD09BB223F400539BB2838170478088C0F30D
S31508008BE0080070470388194201D001207047002009
S31508008BF0704700BF82B00023019300932A4A136886
S31508008C0043F480331360284B1B6803F40033009346
S31508008C10019B01330193009B1BB9019BB3F5A06F20
S31508008C20F1D1214B1B6813F4003F02D001230093B6
S31508008C3001E000230093009B012B32D11A4B1A6CDA
S31508008C4042F080521A6419490A6842F440420A609E
S31508008C509A689A609A6842F400429A609A6842F45E
S31508008C60A0529A60124A5A601A6842F080721A60D4
S31508008C700D4B1B6813F0007FFAD040F205620D4BCE
S31508008C801A60A3F580639A6822F003029A609A68CC
S31508008C9042F002029A60044B9B6803F00C03082B0F
S31508008CA0F9D102B0704700BF00380240007000409A
S31508008CB008544007003C024008B50F4AD2F88830ED
S31508008CC043F47003C2F888300C4B1A6842F001026C
S31508008CD01A60002199601A6822F0847222F48032A0
S31508008CE01A60074A5A601A6822F480221A60D96004
S31508008CF0FFF780FF08BD00BF00ED00E00038024026
S31508008D001030002408B5FFF735FC00F099F808BDC7
S31508008D1008B5FFF7F7FFFFF79FFBFFF74DFCFFF7D7
S31508008D2023FCFAE707498D460749084A084B9A4241
S31508008D30BEBF51F8040B42F8040BF8E70548804714
S31508008D400548004700000220708F00080000002038
S31508008D507C000020B98C0008E98100083349344AB0
S31508008D60002301E041F8043B9142FBD3FFF7D0FF13
S31508008D70FEE7FEE7FEE7FEE7FEE7FEE7FEE7FEE7BD
S31508008D80FEE7FEE7FEE7FEE7FEE7FEE7FEE7FEE7AD
S31508008D90FEE7FEE7FEE7FEE7FEE7FEE7FEE7FEE79D
S31508008DA0FEE7FEE7FEE7FEE7FEE7FEE7FEE7FEE78D
S31508008DB0FEE7FEE7FEE7FEE7FEE7FEE7FEE7FEE77D
S31508008DC0FEE7FEE7FEE7FEE7FEE7FEE7FEE7FEE76D
S31508008DD0FEE7FEE7FEE7FEE7FEE7FEE7FEE7FEE75D
S31508008DE0FEE7FEE7FEE7FEE7FEE7FEE7FEE7FEE74D
S31508008DF0FEE7FEE7FEE7FEE7FEE7FEE7FEE7FEE73D
S31508008E00FEE7FEE7FEE7FEE7FEE7FEE7FEE7FEE72C
S31508008E10FEE7FEE7FEE7FEE7FEE7FEE7FEE7FEE71C
S31508008E20FEE7FEE7FEE7FEE7FEE700007C0000201F
S31508008E30F0000020014B1860704700BFEC000020CE
S31508008E4008B50A4B1B680A4AA2FB03239B09013B88
S31508008E50084A5360F021084B83F8231000209060DD
S31508008E6007231360FFF7E6FF08BD00BF10000020C8
S31508008E70D34D621010E000E000ED00E0014B1868E9
S31508008E80704700BFEC000020024A136801331360E4
S31508008E90704700BFEC00002008B5074B044613B125
S31508008EA00021AFF30080054B1868836A03B1984721
S31508008EB0204600F033F800BF00000000608F00086D
S31508008EC070B50E4B0E4CE41AA41000251E46A5429A
S31508008ED004D056F8253098470135F8E700F020F811
S31508008EE0084C094BE41AA41000251E46A54204D0D6
S31508008EF056F8253098470135F8E770BD740000200C
S31508008F007400002078000020740000200244034604
S31508008F10934202D003F8011BFAE77047FEE7000008
S31508008F20F8B500BFF8BC08BC9E467047F8B500BF48
S31508008F30F8BC08BC9E4670470502060206030703EE
S31508008F400803090309040A040B040C040C050D059F
S31508008F500E050F050F06100610071008430000003F
S30D08008F601400002000000000C7
S30D08008F6880F2FF7F0100000002
S31508008F7000000000010203040102030406070809B1
S31508008F80007A030A0000000000000000000000004C
S31508008F9000000000000000000000000000000000C3
S31508008FA0000000005C8F00080000000000000000C0
S31508008FB000000000000000000000000000000000A3
S31508008FC00000000000000000000000000000000093
S31508008FD00000000000000000000000000000000083
S31108008FE000000000B18100088D81000827
S7050800800072
